:0200000480007A
:100000006F008004732F2034930F80006308FF0378
:10001000930F90006304FF03930FB0006300FF038E
:10002000130F000063040F0067000F00732F2034CC
:1000300063540F006F00400093E19153171F0000BD
:1000400023223FFC6FF09FFF93000000130100008C
:10005000930100001302000093020000130300004C
:100060009303000013040000930400001305000034
:10007000930500001306000093060000130700001C
:100080009307000013080000930800001309000004
:1000900093090000130A0000930A0000130B0000EC
:1000A000930B0000130C0000930C0000130D0000D4
:1000B000930D0000130E0000930E0000130F0000BC
:1000C000930F0000732540F16310050097020000B4
:1000D000938202017390523073500018970200000F
:1000E00093824202739052309B021000939252030B
:1000F0009382F2FF7390023B9302F0017390023AF5
:100100007350403097020000938242017390523046
:10011000735020307350303093010000970200007C
:10012000938282EE73905230130510001315F5017F
:10013000635C05000F00F00F930110009308D005D9
:10014000130500007300000093020000638A0200A0
:1001500073905210B7B200009B82921073902230BD
:100160007350003097020000938242017390123462
:10017000732540F17300203093000000130100004C
:100180003B87200093030000930120006316774C07
:1001900093001000130110003B8720009303200000
:1001A00093013000631A774A930030001301700006
:1001B0003B8720009303A00093014000631E774813
:1001C000930000003781FFFF3B872000B783FFFFCC
:1001D0009301500063127748B700008013010000BC
:1001E0003B872000B70300809301600063167746C9
:1001F000B70000803781FFFF3B872000B783FF7F78
:1002000093017000631A7744930000003781000067
:100210001B01F1FF3B872000B78300009B83F3FFA6
:1002200093018000631A7742B70000809B80F0FF43
:10023000130100003B872000B70300809B83F3FF7E
:1002400093019000631A7740B70000809B80F0FF15
:10025000378100001B01F1FF3B872000B78300803E
:100260009B83E3FF9301A0006318773EB7000080F3
:10027000378100001B01F1FF3B872000B78300801E
:100280009B83F3FF9301B0006318773CB7000080B5
:100290009B80F0FF3781FFFF3B872000B783FF7F04
:1002A0009B83F3FF9301C0006318773A930000002B
:1002B0001301F0FF3B8720009303F0FF9301D00070
:1002C000631C77389300F0FF130110003B87200078
:1002D000930300009301E000631077389300F0FF70
:1002E0001301F0FF3B8720009303E0FF9301F00030
:1002F0006314773693001000370100801B01F1FF73
:100300003B872000B7030080930100016316773418
:100310009300D0001301B000BB8020009303800144
:1003200093011001639A70329300E0001301B00052
:100330003B8120009303900193012001631E7130E3
:100340009300D000BB8010009303A0019301300103
:1003500063947030130200009300D0001301B000CA
:100360003B872000130307001302120093022000B2
:10037000E31452FE9303800193014001631E732C2A
:10038000130200009300E0001301B0003B8720003F
:100390001300000013030700130212009302200051
:1003A000E31252FE93039001930150016316732AE6
:1003B000130200009300F0001301B0003B872000FF
:1003C00013000000130000001303070013021200C3
:1003D00093022000E31052FE9303A00193016001F9
:1003E000631C7326130200009300D0001301B000B9
:1003F0003B8720001302120093022000E31652FEF6
:1004000093038001930170016318772413020000A5
:100410009300E0001301B000130000003B872000B0
:100420001302120093022000E31452FE9303900182
:100430009301800163127722130200009300F00001
:100440001301B00013000000130000003B872000E0
:100450001302120093022000E31252FE9303A00144
:1004600093019001631A771E130200009300D000DD
:10047000130000001301B0003B872000130212009C
:1004800093022000E31452FE930380019301A00124
:100490006314771C130200009300E00013000000B7
:1004A0001301B000130000003B872000130212006C
:1004B00093022000E31252FE930390019301B001D6
:1004C000631C7718130200009300F0001300000073
:1004D000130000001301B0003B872000130212003C
:1004E00093022000E31252FE9303A0019301C00186
:1004F00063147716130200001301B0009300D000BC
:100500003B8720001302120093022000E31652FEE4
:10051000930380019301D00163107714130200004C
:100520001301B0009300E000130000003B8720009F
:100530001302120093022000E31452FE9303900171
:100540009301E001631A7710130200001301B00059
:100550009300F00013000000130000003B87200010
:100560001302120093022000E31252FE9303A00133
:100570009301F0016312770E130200001301B00023
:10058000130000009300D0003B87200013021200EC
:1005900093022000E31452FE9303800193010002B2
:1005A000631C770A130200001301B000130000005F
:1005B0009300E000130000003B87200013021200AC
:1005C00093022000E31252FE930390019301100264
:1005D00063147708130200001301B0001300000039
:1005E000130000009300F0003B872000130212006C
:1005F00093022000E31252FE9303A0019301200214
:10060000631C77049300F0003B0110009303F0009B
:100610009301300263127104930000023B810000D9
:10062000930300029301400263187102BB000000B3
:100630009303000093015002639070029300000145
:100640001301E0013B80200093030000930160024E
:1006500063147000631030020F00F00F638001001C
:100660009391110093E111009308D00513850100C7
:10067000730000000F00F00F930110009308D005E5
:100680001305000073000000731000C0000000009C
:10069000000000000000000000000000000000005A
:1006A000000000000000000000000000000000004A
:0C06B0000000000000000000000000003E
:1010000000000000000000000000000000000000E0
:1010100000000000000000000000000000000000D0
:1010200000000000000000000000000000000000C0
:1010300000000000000000000000000000000000B0
:081040000000000000000000A8
:040000058000000077
:00000001FF
